:030000000219FDE5
:03000B000200A848
:03002B0002015B74
:03005B000202EFAF
:030073000202DCAA
:1000800002030406080C10182030406080040608A3
:100090000C10182030406080A0C00003070F1F051F
:1000A000050D050305030302C2AFC0D0C0E0206206
:1000B00014E5256009E473E525F4F58AD262D0E001
:1000C000D0D0D2AF3285268AC262E526F4603030C5
:1000D000682620720DD0E0D0D0C290C291C292D2D8
:1000E000AF32C290C291C292206F0D20660A740195
:1000F000D5E0FDE57BF45290D0E0D0D0D2AF3275A0
:100100008A00C28DD26201F801B73068052066020C
:10011000D29001B7306805206602D29101B73068ED
:1001200005206602D29201B7D29330680A20660792
:100130007405D5E0FDD29001B7D29430680A2066EC
:10014000077405D5E0FDD29101B7D29530680A2039
:1001500066077405D5E0FDD29201B7C2AFC2AD53B8
:10016000E6EFC0D0C0E0D2D3D2AFC2CEE52A60075E
:10017000207449152A21BC7800790020742EE5806E
:10018000307E01F430E60278FF53DACF207E03435D
:10019000DA20307E0343DA10C2D8C271E580307EA7
:1001A00001F430E60279FFC3E89970CB3061037542
:1001B0002A18207403752A18885CD27020740DE503
:1001C0002B6004152B21CC43DA01C2D820700241E8
:1001D0003FA85C206102C270207431C3E894F040F3
:1001E0000374F0F8E8C4540F28F87984B703024187
:1001F0000CC313C3138721200802C313200A06C3AC
:10020000C898F8410C28F8500374FFF8C3E89565C6
:100210005003E565F88822E52D54066022206B1F07
:10022000E536C333C333F8E564C313C313F9C39589
:100230002240028922E82522F52250037522FF85FB
:100240002224A824C3E52495614002A8618825E5FD
:100250006670024183C3E8AA669A5003E8FAE4F99B
:10026000EAC333FBE568F45B29400D2567F8E567D1
:1002700060021567400B41830AC3E5679A50020587
:100280006778FF8826C26FC3E52694F84002D26FD4
:10029000C3E52594404002D26420CF0AD0E0D0D0FC
:1002A00043E610D2AD32C2CF053A7801E52A6005A7
:1002B000307402152AC3E55C94014005755F004166
:1002C000D2756000756900E55F2401F55F50037524
:1002D0005FFFD0E0D0D043E610D2AD32C2AF53E6DC
:1002E0007F7592FA7593FFC260759104D2AF32C2E6
:1002F000AF53E6EFC2ADC0D0C0E0C0F0D2D3D2AFB2
:10030000A8FBA9FCC2D8307102615653DACF207E17
:100310000343DA10307E0343DA20D271E580307E69
:1003200001F420E602612D88278928A18353DACFC2
:10033000207E0343DA20307E0343DA10C2D8C27134
:10034000307402A16F7800E580307E01F430E6025F
:10035000A16F885CA15753DACF207E0343DA2030A7
:100360007E0343DA10C271206102812F53DACF205D
:100370007E0343DA10307E0343DA20C2D8D271887C
:10038000578958C3E89555F8E99556F97B007E08DA
:100390007A00C3E8948CE994005005755B008121D4
:1003A000882178A2E6A8216055C3E894C8E99400A2
:1003B0005008E4D2E4FB7A0A61FCC3E89468E9944B
:1003C000015008E4D2E3FB7A0F61FCC3E894D0E962
:1003D00094025008E4D2E2FB7A1E61FCC3E894A0C8
:1003E000E994055008E4D2E1FB7A3C61FCC3E8944F
:1003F00098E994085008E4D2E0FB7A787E00C3E8DC
:100400009559FCE9955AFD30E70AECF42401FCED1E
:10041000F43400FD755B00C3EC9AED9E5003755BF0
:10042000018859895A8557558558567802A157C36E
:10043000E89527F8E99528F9307C02A13B307B024A
:10044000A13B307A02A1342075028152E9FDE8FC1B
:100450008171E9C313F9E813F8307902A134E9C3D3
:1004600013F9E813F8307802A134E9C313FDE81357
:0F047000FC20612CC3EC941CED940240028188A7
:10047F00ED701EC3EC94C850180529E529700215BC
:10048F0029C3E529940A5002A16F755C00D270A1AF
:10049F006FE529600215297888E6F97400207F0836
:1004AF007896B90302789EE624FAFEE43400FFC37F
:1004BF00EC9EFCED9FFD9208B90310A20850072097
:1004CF007609D27681DA307602C276A2085016B952
:1004DF00030DECF42401FCEDF43400FD0204F47878
:1004EF00007900A13BB90315EC33FCED33FDC3ECF0
:1004FF00940AFCED9400FD50047C007D00C3EC9445
:10050F00FFED9400400678FF7900A13BEC8572F077
:10051F00A4C5F0A2F733F87900400302055778FF1E
:10052F007900020557E9C313F9E813F8307C0EE997
:10053F00600278FFC3E81338F8E43400F9C3E89495
:10054F00FFE99400400278FF885CD270206102A11D
:10055F006F741FF4552F4BF52FC274EB7002D274CA
:10056F00752A18307403752A0A306102A18320742A
:10057F000353DAFE207403752B06D0F0D0E0D0D0F1
:10058F00D2AD43E6103279010205B379030205B308
:10059F00790A0205B3791E0205B379640205B379AE
:1005AF00C80205B37817E4D5E0FDD8FAD9F6227A58
:1005BF00147B780205DA7A107B8C0205DA7A0D7BD0
:1005CF00B40205DA7A0B7BC80205DA7902E4D29419
:1005DF00D5E0FDD291D5E0FDC291D5E0FDC294D515
:1005EF00E0FDE920E002D29030E002D292E573D52F
:1005FF00E0FDE920E002C29030E002C2927496D58D
:10060F00E0FDD9C9EAF8D5E0FDD8FBDBBED29422D4
:10061F00C37C007D0075F00005F0EA33FAEB33FB85
:10062F0050F6EB13FBEA13FAC3E9FFE8FEE89AF87A
:10063F00E99BF95004EFF9EEF8B3EC33FCED33FD21
:10064F00D5F0DFEDF9ECF822E889F08A20D2D4F862
:10065F00A9F07B0030F70B7BFFF42401F8E9F434A9
:10066F0000F9E88520F0A4ADF0F8E98520F0A4AFFB
:10067F00F0FEED2EF974003FFA7C04C3EA13FAE999
:10068F0013F9E813F8DCF48BF030F70AE8F42401DF
:10069F00F8E9F43400F9E889F0C2D4F8A9F022227D
:1006AF00C3E54113F9E54013F8C3E54498F8E54570
:1006BF0099F9500CC3E89480E994FF40160206E6BE
:1006CF00C3E8947FE9940050030206E6787F79002F
:1006DF000206E6788079FF8849894A22E54925464E
:1006EF00F8E54A3547F9854A20E4300701F43548E3
:1006FF00FA30E709C3EA94F04015020724C3EA94DD
:10070F000F500302072478FF79FF7A0F020724782E
:10071F000079007AF0C3E5249561500AC3740195FE
:10072F0024500B020742E54A20E70E020742E54A32
:10073F0030E706884689478A482278A5E6FAC3E556
:10074F004933F8E54A33F9D157E930E70BC3E89459
:10075F0080E994FF4013E17CC3E8947FE994005053
:10076F0002E17C787F7900E17C788079FFE820E7EF
:10077F0015C3E52398F84009C3E894014003020725
:10078F00A378010207A3E8F424012523F84003020C
:10079F0007A378FF884B2278A6E6FAA847A948D185
:1007AF0057E930E70CC3E89401E994FF40160207BC
:1007BF00D7C3E894FFE9940050030207D778FF7975
:1007CF00000207D7780179FFE920E715C3E54B98B9
:1007DF00F84009C3E8940140030207FE78010207BD
:1007EF00FEE8F42401254BF840030207FE78FF884A
:1007FF00242278FFC26420693D206A12D264C3E5C7
:10080F0041940A4009C3E52594405002C26479A17E
:10081F00E76023E541601F74FF8541F0848539F05F
:10082F00306A0375F005A4F8C5F0600278FFC3E8DD
:10083F0095645002A864886322C3E5409440E54163
:10084F009401E5635003140159046002F563220219
:10085F0008612275E890227883E6FFE5E820ECF73F
:0D086F00A8BDA9BE0570C3E57094084052F5
:10087C00757000E9FA79A0E76044EA7007E57160E9
:10088C001B02089CC3E895716010E5715006600C62
:10089C00140208A80460F90208A8E571F571C39464
:1008AC00F6401B7561C0C394064013756180C394F8
:1008BC0006400B756140C39406400375610075BB1F
:1008CC000E22E561F460020561E570B4070375BBA7
:1008DC001022743279A787F0A4C5F0A2F733F8C3BD
:1008EC00E895614002A8618822882488258826889A
:1008FC0064227540007541F022C2AF75C820A8CCA7
:10090C00A9CDAA3A30CF010A75C824D2AFAB3BAC03
:10091C003C883B893CC3E89BF8E99C206908F9308A
:10092C0067024111216EAD3D8A3DF9EA9DFA6004E2
:10093C0078FF79FFAE3EAF3F8B3E8C3FA83BA93C86
:10094C00C3E89EF8E99FF9C3E54113FBE54013FAB0
:10095C00E82AF540E93BF54150067540FF7541FF2B
:10096C0021B8AA40AB41AC40AD417E047F02C3EB41
:10097C00940440021E1FC3EB940840021E1FC3EDDB
:10098C0013FDEC13FCDEF7C3EA9CFAEB9DFBEF6066
:10099C0009C3E913F9E813F8DFF7EA28FAEB39FB96
:1009AC008A408B4150067BFF8B408B41C3EB9402FA
:1009BC005002D2673069047F0321E37892E6FFC3CB
:1009CC00E537948240110FC3E53794A040010FC363
:1009DC00EF940640027F057E02E541C4540FF9E511
:1009EC0041C454F0F8E540C4540F28F8C3E89EFA0B
:1009FC00E99400FB4009C3EA9402EB940050047A9A
:100A0C0002E4FB415DAA40AB41EBC4FEEAC4540FC7
:100A1C004EFCC3EA9CFAEB9400FBC3E813C313F837
:100A2C00EA28FAEB3400FB8A408B41C3EB9402407A
:100A3C0002C2677802EBC4FE7B00EAC4540F4EFA84
:100A4C00C3EA98FA4005C3940250027A027892E6FF
:100A5C00FF306002415D855192855293D26043E62E
:100A6C0080C3E49AF8E49BF930670241E9E8FAE9BB
:100A7C00FBD3E913FDE813FC88518952C3EF9403AF
:100A8C006038EF20E00DE82CF8E93DF9ECFAEDFBCD
:100A9C00020AB2E828F8E939F9C3E82402F8E93483
:100AAC0000F97AFE7BFFC3EF9403400E8A538B54FC
:100ABC00884D894E8C4F8D50611D885389548A4DB9
:100ACC008B4E8C4F8D503069127553F07554FF75E9
:100ADC004FF07550FF7551F07552FF611DE8FAD358
:100AEC00E813FC8851C3EF94036020EF20E007E883
:100AFC002CF8ECFA6109E8282402F87AFEC3EF948A
:100B0C000340088A53884D8C4F611D88538A4D8C45
:100B1C004FE568C3335002646BF56830600261279F
:100B2C00753402D26043E680E52D54066034A8404B
:100B3C00A941C3E913F9E813F8C3E913F9E813F869
:100B4C00306904E92440F9C2AF53E67F759100C3C4
:100B5C00E498F594E499F595759104D26043E68098
:100B6C00D2AF22D265754300752000306C0375201E
:100B7C0040020B8ED265754300752040306C0375B6
:100B8C00200078017901206720E52D54066002C20F
:100B9C00657914E541C313700104F8C39414400241
:100BAC007814306904781B791B206010E543600CC5
:100BBC00306903D53404D26D8131712F0543E59B27
:100BCC00F45440B52002811B30690908C3E89940F0
:100BDC00011861B520650A08C3E8994002618E616D
:100BEC00B5C265C2AF53E67F75910030671275943C
:100BFC00007595FE759104D26043E680D2AF618E8C
:100C0C00AE40AF41C3E49EF594E49FF5958100C3DB
:100C1C00E53394015002618E306502618ED80281F9
:100C2C002F61B5C26DC2AF53E67F759100855394A9
:100C3C00855495759104854D92854E93D26043E60B
:100C4C0080D2AFE52D54066008206A020533020CF1
:100C5C006D306D0D206C0A2065071581158102150C
:0E0C6C00092278003064053065027801E53712
:100C7A0075F007A4F9E5F028F5F0E9A2F013A2F15E
:100C8A0013A2F213F537C394785003753778C3E586
:100C9A003795384008D266C290C291C2923060023B
:100CAA0081A7854F92855093D26043E68022207DAA
:100CBA0016C2AF754202D294C293306202D292D265
:100CCA00AF759F11020EA7C2AF754202D294C295A8
:100CDA00306202D290D2AF759F11020EA7307243D2
:100CEA00207D20C2AF754203900139757B10C292F4
:100CFA00D295306204D291A105C294D2AF759F01F8
:100D0A00020EA7C2AF754203900139757B10C290DB
:100D1A00D293306204D291A125C294D2AF759F2199
:100D2A00020EA7207D17C2AF754203900114C2922A
:100D3A00306202D291D2AF759F01020EA7C2AF757F
:100D4A004203900114C290306202D291D2AF759FD1
:100D5A0021020EA7207D16C2AF754204D293C29516
:100D6A00306202D291D2AF759F21020EA7C2AF752F
:100D7A004204D295C293306202D291D2AF759F01DA
:100D8A00020EA7307243207D20C2AF754205900142
:100D9A0028757B08C291D294306204D290A1ABC26A
:100DAA0093D2AF759F11020EA7C2AF75420590018B
:100DBA004A757B20C291D294306204D292A1CBC2EE
:100DCA0095D2AF759F11020EA7207D17C2AF75424B
:100DDA000590010AC291306202D290D2AF759F117A
:100DEA00020EA7C2AF75420590011EC2913062EB96
:100DFA00D292D2AF759F11020EA7207D16C2AF758F
:100E0A004206D295C294306202D290D2AF759F0147
:100E1A00020EA7C2AF754206D293C294306202D2C2
:100E2A0092D2AF759F21020EA7307243207D20C255
:100E3A00AF75420190014A757B20C290D29330620D
:100E4A0004D292C151C295D2AF759F21020EA7C298
:100E5A00AF754201900128757B08C292D295306223
:100E6A0004D290C171C293D2AF759F01020EA7201E
:100E7A007D17C2AF75420190011EC290306202D244
:100E8A0092D2AF759F21020EA7C2AF75420190019F
:100E9A000AC292306202D290D2AF759F01C2662214
:100EAA00900108757B00C290C291C292D293D294EB
:100EBA00D295C26222788076FF0876FF0876FF080C
:100ECA0076FF08760308760408760B087603087618
:100EDA0001087601788C76010876FF0876FF087695
:100EEA00FF0876FF0876FF0876030876FF0876FF84
:100EFA000876FF0876250876D00876FA0876FA0882
:100F0A0076040876FF08760108760008767A08766D
:100F1A00FF0876010876010876000876030876004D
:100F2A00227887E6FFC272BF0302D2727888E6C3CC
:100F3A0094036008C27DE630E102D27DC27E7889E0
:100F4A00E630E102D27EC3EF94026008758E01D2C8
:100F5A0073020F63758E00C273227880E6149000C4
:100F6A00809378A5F67881E6149000809378A6F6A7
:100F7A007886E61490008D9378A7F67886E6F53998
:100F8A00C394025003753902789CE67538FFB4029F
:100F9A00037538A0B4030375388278A3E614900069
:100FAA009A93F566D1AA22227896E6FA7897E6FB12
:100FBA007888E6B40305C3EB940EFB307F047A000D
:100FCA007BFFC3EB9AFCC3948250027C8275720049
:100FDA000572EC8572F0A4C3E5F0947D40F222D24A
:100FEA007FF1B21205A47A007B007C1012059AE503
:100FFA005C2AFA74003BFBDCF37C04C3EB13FBEAC8
:10100A0013FADCF7FEC27F120FB222E5EF20E603E5
:10101A007520000520903FFFE520146006901DFF13
:10102A001460009304600375EF1053D9BF7581C033
:10103A0043FF8012059575EF0043B203E5B324021E
:10104A0020E70DF521E5E320E0068521B343E3011E
:10105A00120EAA7580FF75A40075F1D075D4BF75FC
:0E106A00907875A53F75F2BF75D54075A6014B
:1010780075E241120EAAE4F8F6D8FD756801120E61
:10108800BF12155A78988673753001C2AF1205AE33
:101098001205BE1205A41205C51205A41205CC122C
:1010A80005A41216731205AE1205AE1205A9C2AF39
:1010B80078FA79FA308607D9FBD8F7021C00120FA4
:1010C8002B120F64120FB1120FB278988673120E9A
:1010D800AA75881075890275C82475910475D84059
:1010E80075A82275B80275E690759B80759D007588
:1010F800D10775BC5875BB0E75BA1175E880120515
:1011080095D2AF12085E75360053DACF207E0343BE
:10111800DA20307E0343DA1043DA01C2D8C27112F2
:1011280005AED2617B037A0CE55B70077A0CDB03B2
:101138000210B61205A42070030210B6C270E55C56
:10114800C3940240E1E52F541F855E5DF55EB55DF1
:10115800D5DAD5C26153DACF207E0343DA20307E58
:101168000343DA10C2D8C27178A2E67008D274E5D7
:101178002F54E0F52FC2757529001205A93074099E
:10118800C3E529940A4002D27512059A7802307490
:10119800027800C3E55C9840F0C2AF1205BE1205A4
:1011A800BE1205BED2AF1205AE754C007888E6B403
:1011B8000302419912059A788CE6C3940150030200
:1011C8001299E530C394015003021299207435C373
:1011D800E55C94FF5003021299C2AF1205D3D2AF57
:1011E8001205A9C3E55C940150EFC2AF1205BE1207
:1011F800059F1205BED2AF1205A9C3E55C94FF4056
:10120800E90216F87F05D27F120FB21205A9C2AF04
:10121800C27F120FB2AE5CC3E55C947FD2AF407B55
:10122800120595C2AF1205D3D2AFDFDA120FE9C3A8
:10123800EE94057897F61205AE12159C12167B7F70
:101248000AD27F120FB21205A9C2AFC27F120FB223
:10125800AE5CC3E55C947FD2AF50E4120595C2AF93
:101268001205BE12059F1205BED2AFDFD4120FE9D8
:10127800EE24037896F61205AE12159C1216AA12E1
:1012880005A9120FB2C3E55C94FF500221D40216DF
:10129800F8C3E55C954C4003855C4C1205A97801C0
:1012A8007988E7B403027805C3E55C98400221B465
:1012B800C2AF1205D31205D31205D3D2AF1205AEB1
:1012C800753000E4F531F5320531E531F4703F054C
:1012D80032789AE67819146012783214600D787DA5
:1012E80014600878FA146003753200C3E532984038
:1012F8001D120EAA1205951532753100789986735C
:10130800C2AF1205D3D2AF789886731205A9120519
:101318009FE52A700530740201B6780120740278BE
:1013280006C3E55C9840A17888E6C394036003127D
:1013380005A9E52A70030210B6C2AF120EAAE4F599
:1013480022F523F524F525F526F567D2AF7885E64D
:10135800C333F565E4F544F545F546F547F548F535
:1013680070F52CF52DF53775700875BB10120595BD
:10137800120862E5E820ECFBA8BDA9BEE97001F8F7
:10138800887112086675700875BB10120F2BC2AFF2
:101398007561FF1208DE852261852262852263D28B
:1013A800AF752201752401752501752601856069CF
:1013B800756A017888E6B40307C27D307602D27D6B
:1013C800D268D269753300120E04120E331208FE69
:1013D8001209051208FE1209051208FE120B8012E6
:1013E80006AE120C6E120CB8120905120B6F306E95
:1013F800031206AF2067031208013067031208487A
:10140800120C6E120CE7120905120B80306E0312D3
:1014180006EB120C6E120D5E120905120B6F306E80
:1014280003120749120C6E120D8D120905120B805A
:10143800306E031207A6120C6E120E041209051262
:101448000862120B6F120C6E120E33120866120924
:101458000530692F856461856462856069756A01F4
:0E14680079187A0CC3E53399400CC269D26A38
:101476008A357561FF02148BC3E55C940140030253
:1014860013E4021511306A1D206C1AE53514700636
:10149600C26AD26B61E4F535C3E55C940140030290
:1014A60013E4021511753600788279A4E760027894
:1014B60003C3E55F985054307404E52A604D78887C
:1014C600E6B40317207D0520760781E13076028198
:1014D600E1206C07D26C856461812378F0306C055D
:1014E6008564617820C3E54198500261E4306C1B45
:1014F600C26CC27D307602D27DD26A7535128564A1
:101506006161E40536E55C6002A114753600C2AF80
:10151600120EAA7887E6FE7602120F2B7887EEF671
:10152600E4F522F523F524F525F526F565752C0059
:10153600752D00D2AF1205A9120EAA78A4E6600690
:10154600D290D291D292307409C3E5369404400207
:1015560001B641CB901A0D78201215DEE520B45A5B
:101566000CA31215DEE520B4A50302157C120EBFEE
:1015760012159C02159B901A0378807B0A1215DEC1
:10158600A308DBF9901A0F788C7B191215DEA308D5
:10159600DBF9901A2822C2AF12161D1215F7901AFF
:1015A60000740E1215E3A374061215E3A374151244
:1015B60015E3901A0378807B0A1215E2A308DBF97B
:1015C600901A0F788C7B191215E2A308DBF9121614
:1015D6003012160E901A2822E493F622E6438F0163
:1015E600538FFD75EF0275B7A575B7F1F0538FFEF2
:1015F60022438F02438F0175EF0275B7A575B7F1C8
:10160600901A0DF0538FFC22901A0D745AB1E39084
:101616001A0E74A5B1E3227A3079D07820901A4058
:10162600B1DEE520F709A3DAF7227A3079D0901AED
:1016360040E7B1E309A3DAF922AB74A875BB01024E
:101646007984BB02027985BB03027986BB040279E1
:1016560092BB05027987BB060279A3BB0702799C78
:10166600BB08027988BB09027989E8F7227C051252
:1016760005AEDCFB22C2AF1205BE1205C51205CCB3
:101686001205D312059F1205BE1205C51205CC120E
:1016960005D312059F1205BE1205C51205CC12050B
:1016A600D3D2AF22C2AF1205D31205CC1205C51292
:1016B60005BE12059F1205D31205CC1205C51205EB
:1016C600BE12059F1205D31205CC1205C51205BE22
:1016D600D2AF22AE74AF75C2AF1205BE1205BE12EE
:1016E60005BE12059FDEF21205D312059FDFF8D262
:1016F600AF22D17BD173D17375740175750175767F
:1017060000D1D97C05AD5C1205AEC3ED955C70F5D4
:10171600C3E55C9401400AC3E55C94FF40320217BE
:1017260034D13FB19CD17BC2AF75EF10D173DCD5FC
:101736000576C3E5769403500280C6D1730575E538
:10174600741490009F93F808C3E57598500280AE14
:10175600D173D1730574C3E574940A5002809C1248
:0B1766000EBFB19CC2AF75EF10D17335
:0319FD00021015C0
:101A00000E0615FFFFFFFF03040B0301015AA5019A
:101A1000FFFFFFFFFF03FFFFFF25D0FAFA04FF01DE
:091A2000007AFF0101000300FF40
:101A40002353757065726D6963726F33703541230E
:101A500023424C48454C4923463333302320202031
:101A60002020202020202020202020202020202076
:101C0000C2AFC2D353D9BF7581C043B20343FF8073
:101C1000752438752503B1C975EF0275E24043F1AB
:101C20004053A4BF75D4FFD2867DFA780379E67C51
:101C300010752200752300901DD67B0675249875BB
:101C400025013086028142208608D8FBD9F9DCF7CD
:101C500081B4308608D8FBD9F9DCF781B4B189E4C6
:101C600093A3C39A6004DDC381B4DBDBB17B600264
:101C7000812B7B08E493FAA3B15CDBF87A30B15C8A
:101C8000752200752300B17BEAFCEBFDC3ED94FEE9
:101C9000400EB17B8A278B28ED30E0048A828B834B
:101CA000B17B7AC270D8C3ED94FE601350CEBD00F4
:101CB00025EC60097520007521FF0200008100A855
:101CC00027A9280809D804D90281D3B17FEA89AAB3
:101CD000F281C50D81A0C3ED94035049EDA2E092BD
:101CE000007AC5C3E5829400E583941C50902000DF
:101CF00010438F02438F0175B7A575B7F1F030001F
:101D00001FA827A9280809438F01538FFDD804D99C
:101D100002A12089AAE275B7A575B7F1F0A3A10DBC
:101D2000538FFC817C7AC1BD030CE493A3FAB140CC
:101D3000DCF8B138817C817EAA22AB23B15CEBFA5E
:101D4000EA6222752608C3E52313F523E52213F57D
:101D50002250066323A0632201D526EAB1C9B1C986
:101D600075260AEAF4200102D286300102C286B149
:101D7000C9C3134002C201D526EB22B17FEAFB2082
:101D80008602A17F308602A184752608AE24AF2585
:101D9000C3EF13FFEE13FEB1CDB1C9C3EA13308612
:101DA000024480FA30E703632201C3E52313F523DD
:101DB000E52213F52250066323A0632201D526D91C
:101DC000E52265236523F52222AE24AF250E0FDE22
:101DD000FEDFFCD20122424C48656C693437316326
:041DE000F3300601D5
:00000001FF
